:100000000AC018951895189518951895189518956B
:100010001895189518958FED8DBFC0ECE0EB4E2E1E
:10002000DD275D2EEEE7F0E0A0E6B0E088278D93B7
:100030003197E9F78FEC89B988E18AB9662400E045
:1000400010E820E030E0A0E60D931D932D933C9343
:100050008FEF87BB80E088BB8EEF81BB83EF82BBD5
:1000600088EC90E07CD1B1D094989598969806D081
:1000700081E090E074D1FBCFF894FFCF37D1A5E6B3
:100080008C9300916500003009F492C081E4482F00
:1000900000916500041709F003C08BD0C09A089541
:1000A00082E4482F00916500041709F003C081D055
:1000B000C19A089583E4482F00916500041709F060
:1000C00003C077D0C29A089584E4482F0091650058
:1000D000041709F003C06DD0C39A089585E4482F32
:1000E00000916500041709F003C063D0C49A089515
:1000F00086E4482F00916500041709F003C059D029
:10010000C59A089587E4482F00916500041709F007
:1001100003C04FD0C69A089588E4482F0091650027
:10012000041709F003C045D0C79A089588E5482F01
:1001300000916500041709F005C03BD0949895988C
:100140009698089581E3482F00916500041709F0FF
:1001500002C0949A089582E3482F00916500041725
:1001600009F002C0959A089583E3482F0091650035
:10017000041709F002C0969A089586E3482F00916B
:100180006500041709F002C09498089587E3482F8A
:1001900000916500041709F002C09598089588E35E
:1001A000482F00916500041709F002C09698089541
:1001B0000895C098C198C298C398C498C598C69825
:1001C000C79831E0A5E6B9D00895C09A80E590E0DF
:1001D000C6D0C09880E590E0C2D0C19A80E590E09A
:1001E000BED0C19880E590E0BAD0C29A80E590E098
:1001F000B6D0C29880E590E0B2D0C39A80E590E096
:10020000AED0C39880E590E0AAD0C49A80E590E093
:10021000A6D0C49880E590E0A2D0C59A80E590E091
:100220009ED0C59880E590E09AD0C69A80E590E08F
:1002300096D0C69880E590E092D0C79A80E590E08D
:100240008ED0C79880E590E08AD0949A80E590E0BF
:1002500086D0949880E590E082D0959A80E590E0F1
:100260007ED0959880E590E07AD0969A80E590E0EF
:1002700076D0969880E590E072D0C09A08952020BC
:100280005472616E736D6974746572202D205265AD
:100290006D6F746520416E74656E6E612053776971
:1002A000746368204F76657220436F61782028520E
:1002B00041534F432920402052573358412020209A
:1002C000687474703A2F2F6F6478632E72752F7173
:1002D00072752F686172642F7261732F7261735F20
:1002E00076312E68746D6C202020000088275F9B7B
:1002F000089500C00F931F932F933F93AF93BF9325
:10030000A0E60D911D912D913D915F9B01C00BC009
:100310008827802B812B822B832B39F001501040B2
:1003200020403040F2CF8CB101C08827BF91AF91FF
:100330003F912F911F910F9108958D9103D03A9580
:10034000E1F708955D9BFECF8CB908953197F1F7E1
:100350000895689462F80895E89462F80895EF9318
:10036000FF93EE27E82BE92B31F0EAEFF0E031972D
:0C037000F1F70197D1F7FF91EF9108958C
:00000001FF
